:100000009E014D299E169E1E9E129E190B289E151E
:1000100044200318322808308F0058208E0D8F0B93
:100020000D289E1E3D2062205E209E1A3220372021
:100030000E08031048299E169E1E9E121E19252882
:10004000FE399F001E15031048291E1A2D28920004
:100050001E1644200318322812084B200318322899
:100060009E1E48293D2062201E111E129E1122084C
:100070008400200884178004432822088400200973
:100080008005841780050800372062203D205E200F
:100090001F089E1901388E0008308F008E0D03183E
:1000A0003720031C3D2062205E208F0B4E28372016
:1000B00062202208840020080005FF3E23088400F7
:1000C000210940282308840021083A2804089200C6
:1000D0002208840080309F05083093000310031825
:1000E0009F0A8020920C930B6F280000971A1F0C18
:1000F00080204B21031480201B088F001A08D3286E
:100100008413971F8F2800082004171F20068000E3
:10011000841700082004031C200680009A28000889
:100120002004031C2006171B2006800084172009CA
:1001300080059A2817081F39FF3E8D001608F53EE6
:1001400003188D0A0000E0289F13150803199F1754
:100150000530940027308F001030BA2003308F0014
:10016000E830BA208F016430BA208F010A30BA20FB
:100170001008C1288E0011088D0010088C00112174
:100180000C088C00940303199F1315080319CB283E
:100190001402031808000C08031D9F139F1B08007E
:1001A000303E43298F018E00FF308E07031C8F07DE
:1001B000031C482903308D00DF30E020D4288D0156
:1001C000E83E8C008D09FC30031CE9288C070318DD
:1001D000E6288C0764008D0FE6280C18EF288C1C8D
:1001E000F3280000F3280800013E93000A308E0037
:1001F0008F011121930BF928100808008E0001309F
:10020000012994000F080D02031D08290E080C0295
:10021000043003180130031902301405031DFF30A8
:10022000482991019001103092000D0D900D910D13
:100230000E0890020F08031C0F0F910203182729C4
:100240000E0890070F0803180F0F910703108C0D6D
:100250008D0D920B15290C084829103094008D0142
:100260008C01930C920C031C3B290E088C070F0881
:1002700003180F0F8D078D0C8C0C910C900C940BA8
:1002800031291008482984001D088A001C088200B2
:10029000831303138312640008008316850113304F
:1002A0008600831285018601552985018601861203
:1002B0008316861264308312D2206400061E182A28
:1002C0000130A800A90128088C0029088D008F01A1
:1002D0001E30FE20031D75296400061E182A643096
:1002E000D220A80A0319A90F63298616831686123D
:1002F000831213308F008830D32086128316861223
:1003000083120530A2000430A0000530A30008309D
:10031000A100A0301D20FF301D20DC301D20042056
:10032000A7000220A6000A30D2200130AA00AB01AB
:100330000230A400A50124088C0025088D002708A0
:100340008F002608FE20031D0B2A0530A200043072
:10035000A0000530A3000830A100A0301D20250812
:100360001D2024081D200420AD000220AC000A300E
:10037000D2202C088C002D088D0064308E008F0157
:100380001121B5002C088C002D088D000130F420BF
:10039000B4002C088C002D088D000030F420B30030
:1003A0000630A2000230A0005430960097019A0156
:1003B0009B0195012A0890002B08910066309C0053
:1003C0009D01A4202C3067209501350890009101F3
:1003D00066309C009D01A4202E30672095013408D2
:1003E0009000910166309C009D01A4209501330886
:1003F0009000910166309C009D01A4200D30672083
:100400000A306720AA0A0319AB0A0230A407031CAA
:100410009B29A50F9B2986168316861264308312AA
:10042000D22086128316861264308312D2200B2AC1
:100430000130AA00AB010130A800A90128088C00F6
:1004400029088D008F012830FE20031D372A8616CB
:100450008316861264308312D22086128316861287
:1004600064308312D220A80A0319A90F1E2A64003F
:100470000618372A86168316861283120B308F00D1
:10048000B830D32086128316861283122C30AC002B
:100490000130AD002C088C002D088D00EA308F0053
:1004A0005F30FE20031D842A6400061C892AF83070
:1004B000DF206400061C892AF830DF206400061C57
:1004C000892AF830DF206400061C892AF830DF20F2
:1004D0000430D2206400061C892AF830DF20640032
:1004E000061C892AF830DF206400061C892AF830AF
:1004F000DF206400061C892AF830DF200430D22077
:10050000AC0A0319AD0F4A2A0B308F00B830D32044
:10051000462A86168316861283122A0892002B0812
:10052000930002308E008F012D21A4001108A50038
:100530002C088C002D088D0064308E008F01112155
:10054000B3002C088C002D088D000130F420B4007D
:100550002C088C002D088D000030F420B5000630EA
:10056000A2000230A0005430960097019A019B012E
:1005700095012A0890002B08910066309C009D018F
:10058000A4202C306720950133089000910166303B
:100590009C009D01A4202E30672095013408900016
:1005A000910166309C009D01A420950135089000C2
:1005B000910166309C009D01A4200D3067200A3017
:1005C00067200530A2000430A0000530A3000830E9
:1005D000A100A0301D2025081D2024081D202D0865
:1005E0001D202C081B200A30D2200530A200043028
:1005F000A0000530A3000830A100A0301D20FF306E
:100600001D20DC301D2025081D2024081B200A3059
:10061000D220AA0A0319AB0A0B308F008F30D320E7
:0E0620008612831686128312462A6300152B5B
:02400E00F53F7C
:00000001FF
